:020000040000FA
:060000000219FD0200C818
:03000B0002008D63
:03002B000200923E
:03005B000202C6D8
:030073000200B5D3
:100080000406080C10182030406080A0C0C28D0506
:100090004032C0D0C0E0C2CF0541E5646009E563ED
:1000A000600575630001B0756301E52360021523E7
:1000B000D0E0D0D032C2AF53E67F7592FA7593FF8D
:1000C000C22053917FD2AF32C0D0C0E0C0F0D2D3B3
:1000D0005388EFA88AA98CAA40308D010A758A003E
:1000E000758C00754000438810E564700AC3E833DE
:1000F000F8E933F9EA33FA30331FE8C4540FFAE968
:10010000C454F04AFAC3132AFAC3E833F8E933F9BE
:10011000E82AFAE93406FB216C30320FC3E833E9F0
:1001200033FAE82AFAE93400FB216C303115E8751E
:10013000F056A4AAF0E975F056A42AFAC5F03400E6
:10014000FB216CC3EA13FAE913F9E813F8E875F038
:1001500056A4AAF0E975F056A42AFAC5F03400C3F3
:1001600013FBEA13FAC3EB13FBEA13FAC3EB941283
:100170005006C3EB9406501A0522E52270021522A0
:10018000C3E522940A500241BC7552007A007B00FC
:10019000418DE522600215223035067C007D082164
:1001A000ACAC31AD32303A04AC33AD34C3EA9CFA76
:1001B000EB9DFB9208AE5EAF5F303A4250072034B1
:1001C00009D23421CA303402C234303404AE60AFB4
:1001D00061203902B234C3EA33FAEB33FBA2085090
:1001E0000AEAF42401FAEBF43400FBC3EA9450FA6F
:1001F000EB9400FB501478007A007B00410AA208BF
:10020000500878007A007B004169E5255403601BA3
:10021000202A18E55B33F9EB7007C3E99A4002E93D
:10022000FAE53CC4332AFAEB3400FBEA8EF0A4F979
:10023000AAF0EB8EF0A42AFAC5F03400FBC3EB134E
:10024000FDEA13F8C3ED13FDE813F80FEF14600493
:10025000C3E833F8C3E933EA33FAEB33FBDFEDEB02
:1002600030E30678FF7AFF7B078852D230C3E894E8
:10027000404002D221C3E559FC955A4003AC5AC311
:10028000EC95525008EC75F008A4FAABF0EAF4F8DB
:10029000EBF45407F9C3E89464FAE99400FB5004C2
:1002A0007A007B00885489558A568B5775230AD06B
:1002B000F0D0E0D0D053F7DF43F7403275230AD0B7
:1002C000F0D0E0D0D032C0D0C0E0D2D3A8F9E55809
:1002D00030E107E5FA30E2076114E5FA30E235C3B0
:1002E000E55513F8E55413F5FB88FCC3E55713F8FF
:1002F000E55613F5E988EA85555853F7BFC3E5522B
:10030000940140057553006114E5532401F55350E1
:10031000037553FF53F7DFD0E0D0D032790180145A
:1003200079038010790A800C791E80087964800432
:1003300079C880007817E4D5E0FDD8FAD9F6227A9A
:10034000147B7880127A107B8C800C7A0D7BB480C1
:10035000067A0B7BC880007902E4C293D5E0FDD217
:1003600092D5E0FDC292D5E0FDD293D5E0FDE92023
:10037000E002D29030E002D294E562D5E0FDE920BF
:10038000E002C29030E002C2947496D5E0FDD9C973
:10039000EAF8D5E0FDD8FBDBBEC2932278FFC2218C
:1003A00020283D202912D221C3E548940A4009C3E0
:1003B000E55294405002C22179A1E76023E54860EC
:1003C0001F74FF8548F084853FF030290375F005E0
:1003D000A4F8C5F0600278FFC3E8955B5002A85B03
:1003E000885A22C3E54794A0E5489400E55A500393
:1003F0001461F4046002F55A2275E89022055CC38A
:10040000E55C94084055E5E820ECF2A8BDA9BE756E
:100410005C00E9FA79A0E76041EA7006E55D6018E2
:10042000800CC3E8955D600EE55D5005600A1480A0
:10043000070460FA8002E55DF55DC394F6401B7524
:1004400059C0C394064013755980C39406400B7578
:100450005940C39406400375590022E559241050B1
:100460000274FFF55922743279A687F0A4C5F0A270
:10047000F733F8C3E895594002A859885B227547BD
:10048000007548F022C2AF75C800A8CCA9CDAA411A
:1004900030CF010A75C804D2AFC3EA13FAE913F9E1
:1004A000E813F8AB42AC4388428943C3E89BF8E9C0
:1004B0009C20280A547FF9302C02A19F81FCAD4476
:1004C0008A44F9EA9D547FFA600478FF79FFAE45CB
:1004D000AF468B458C46A842A943C3E89EF8E99FE6
:1004E000F9C3E54813FBE54713FAE82AF547E93B6A
:1004F000F54850067547FF7548FFA146AA47AB4827
:10050000AC47AD487E047F02C3EB9404400A1E1F33
:10051000C3EB940840021E1FC3ED13FDEC13FCDE79
:10052000F7C3EA9CFAEB9DFBEF6009C3E913F9E816
:1005300013F8DFF7EA28FAEB39FB8A478B485006B5
:100540007BFF8B478B48C3EB94025002D22C3028A0
:10055000047F03A1717892E6FFC3E53D94824011C8
:100560000FC3E53D94A040010FC3EF940640027F06
:10057000057E02E548C4540FF9E548C454F0F8E597
:1005800047C4540F28F8C3E89EFAE99400FB4009D9
:10059000C3EA9401EB940050047A01E4FBA1EBAAB6
:1005A00047AB48EBC4FEEAC4540F4EFCC3EA9CFAC6
:1005B000EB9400FBC3E813C313F8EA28FAEB34000A
:1005C000FB8A478B48C3EB94024002C22C7802EBB3
:1005D000C4FE7B00EAC4540F4EFAC3EA98FA400501
:1005E000C3940150027A017892E6FF30200280FB2A
:1005F000854E92854F93D22043E680C3E49AF8E477
:100600009BF9C3E833F8E933F9302C02C17DE8FAED
:10061000E9FBD3E913FDE813FC884E894FC3EF943F
:10062000036037EF20E00CE82CF8E93DF9ECFAED37
:10063000FB8013E828F8E939F9C3E82401F8E93424
:1006400000F97AFF7BFFC3EF9403400E8A508B5171
:10065000884A894B8C4C8D4DC1B1885089518A4A4A
:100660008B4B8C4C8D4D3028127550F07551FF75A9
:100670004CF0754DFF754EF0754FFFC1B1E8FAD3E0
:10068000E813FC884EC3EF94036020EF20E007E8F6
:100690002CF8ECFAC19DE8282401F87AFFC3EF9406
:1006A0000340088A50884A8C4CC1B188508A4A8CD1
:1006B0004C302002C1B1753A02D22043E680E525D4
:1006C0005403602DA847A948C3E913F9E813F8308B
:1006D0002804E92440F9C2AF53E67F759100C3E4D2
:1006E00098F594E499F595759104D22043E680D26B
:1006F000AF22D222754900752000302B03752040AF
:10070000800ED222754900752040302B03752000E1
:1007100078017901202C20E52554036002C222795A
:1007200014E548C313700104F8C39414400278140C
:10073000302804781B791BC3E833F8C3E933F92068
:100740002010E549600C302803D53A04D224E1C7D3
:10075000D1B90549E59B5440B52002E1B1302809E3
:1007600008C3E899400118E13F20220A08C3E8992C
:100770004002E110E13FC222C2AF53E67F75910013
:10078000302C127594007595FC759104D22043E6C7
:1007900080D2AFE110AE47AF48C3EE33FEEF33FF78
:1007A00050047EFF7FFFC3E49EF594E49FF595E13E
:1007B00089C3E53994015002E110302202E110D8DA
:1007C00002E1C5E13FC224C2AF53E67F75910085C7
:1007D0005094855195759104854A92854B93D2200A
:1007E00043E680D2AFE5255403600720290205398E
:1007F000801030240D202B0A20220715811581023C
:100800000F162278003021053022027801E53D756F
:10081000F007A4F9E5F028F5F0E9A2F013A2F1132E
:10082000A2F213F53DC394785003753D78C3E53DBE
:10083000953E400BD223C290C292C29475D57F30B0
:10084000200280FB854C92854D93D22043E6802286
:10085000203810C2AFC293D29175D54FD2AF759FD9
:10086000202124C2AFC293D29575D57CD2AF759F9B
:10087000202124203811C2AFC29475D573D291D2F1
:10088000AF759F30020924C2AFC29075D573D2955F
:10089000D2AF759F10020924203810C2AFC291D286
:1008A0009575D573D2AF759F108079C2AFC295D2BE
:1008B0009175D573D2AF759F308069203811C2AF62
:1008C000C29275D57CD295D2AF759F20020924C201
:1008D000AFC29275D54FD291D2AF759F2002092435
:1008E000203810C2AFC295D29375D57CD2AF759F18
:1008F000308031C2AFC291D29375D54FD2AF759FC0
:10090000108021203810C2AFC29075D54FD293D23B
:10091000AF759F10800EC2AFC29475D57CD293D2B2
:10092000AF759F30C22322C290C292C294C291C2BC
:1009300093C29575D57F22788076FF0876FF08767A
:10094000FF0876FF0876FF0876FF0876090876FF2D
:10095000087601788C76010876FF0876FF0876FF26
:100960000876FF0876FF0876030876FF0876FF080A
:1009700076FF0876250876D008762808765008761F
:10098000040876FF0876020876FF08767A0876FF74
:100990000876010876010876FF0876FF08760008D9
:1009A000760022FA75F00CA4ABF0EAC333F87401B8
:1009B00033F9E8C333F8E933F9E8C32BF8E9340035
:1009C000F9E8C333F8E933F9227888E6C39403D20F
:1009D0003A5002C23AC238E630E102D238A2389226
:1009E000397886E6149000809378A6F67886E6F546
:1009F0003FC394025003753F02789CE6753EFFB4F6
:100A00000203753EA0B40303753E827896E631A3D7
:100A100088318932789EE631A3883389347897E625
:100A200031A3883589363127223035117A007B0091
:100A30007CFF7D007E0051908B5F8A5E22303A22DF
:100A40007896E6FA7B00789EE6FC7D00C3EA33FAEE
:100A5000EB33FBC3EC33FCED33FD7E0A51908B612D
:100A60008A607896303A02789EE6FA7B007897E6BC
:100A7000FC7D007E00303A10C3EA33FAEB33FBC34F
:100A8000EC33FCED33FD7E0A51908B5F8A5E2222AF
:100A9000C3EC9EFCED9400FDC3EC9AFCED9BFDC302
:100AA000EC9423ED940050047C237D00C3EC94FF70
:100AB000ED940140047CFF7D017BFF0B7A000AEA84
:100AC0007009C3EC33FCED33FD41BBEC8AF0A4AEFE
:100AD000F0ED8AF0A42E947C40E4EAF460DD22D2AA
:100AE0003551291203287A007B007C10120320E57F
:100AF000522AFA74003BFBDCF37C04C3EB13FBEAE1
:100B000013FADCF7FFEB60027FFFC2355129227830
:100B1000A5E6F95403D2867002C286E9540CD28746
:100B20007002C287E95430D2967002C296E954C06E
:100B3000700022E5EF20E6037520000520903FFFBE
:100B4000E520146006901DFF146000930460037597
:100B5000EF127597DE7597AD7581C043FF80120364
:100B60001C75EF0275A900312775803F75F1F0758E
:100B7000A4C075803F75D4FF75900075F27F75A590
:100B80007F75900075D57F75A60175E34075E2020B
:100B9000C290C292C29412032CD291D293D29512D7
:100BA000031CC291C293C2953127E4F8F6D8FD31F7
:100BB00037F15778988662753001C2AF1203301250
:100BC000033F12032812034512032812034B12039A
:100BD00028710FC2AF78FA79FA308507D9FBD8F7B8
:100BE000021C0031C9512978988662312775A913F2
:100BF00075A71075C10075A70075640075E40575CB
:100C00008811758E0475890975C80475910475D8A5
:100C10004075D90875F782759E0375960275DA429C
:100C200075DB4275A82375E69075F310759B80758A
:100C30009D0075D12C75BCC075BB1075E88075B270
:100C40000112031CD2AF753C00C230120330C23116
:100C500075220012032CC3E522940A4024D231C22B
:100C60003275220012032CC3E522940A4013D232BB
:100C7000C23375220012032CC3E522940A4002D22B
:100C800033120320203003020BD3C2AF12033F12F2
:100C9000033F12033FD2AF120330303A02A12D12AC
:100CA0000320788CE6C394015002A12DE530C39453
:100CB000015002A12D7F02D235512912032CC2AF5F
:100CC000C2355129AE52C3E552947FD2AF405E1275
:100CD000031CC2AF120351D2AFDFDC51DFC3EF7888
:100CE00097F6120330F1911210397F0AD23551294B
:100CF00012032CC2AFC2355129AE52C3E552947FC4
:100D0000D2AF50E612031CC2AF12033F12032412EB
:100D1000033FD2AFDFD651DFEF24037896F61203FC
:100D200030F19112106812032C512961D312032C57
:100D30007801303A027805C3E552984002819AC2A0
:100D4000AF120351120351120351D2AF1203307587
:100D50003000E4F537F5380537E537F4703E0538EF
:100D6000789AE67819146012783214600D787D1440
:100D7000600878FA146003753800C3E53898401CA1
:100D8000312712031C153875370078998662C2AF77
:100D9000120351D2AF7898866212032C120324E515
:100DA00023700261D37801C3E5529840AA12032C44
:100DB000E5237003020BD3C2AF3127E4D2AFE4F5D1
:100DC0005CF524F525F53D755C0812031C1203F94A
:100DD000E5E820ECFBA8BDA9BEE97001F8885D122A
:100DE00003FD755C08C2AF7559FF120466855B5937
:100DF000855B5AD2AF75A71075C13075A70075A96C
:100E000003756401303A07C238303402D238D22830
:100E100075390011E0310312047E12048512047E3C
:100E200012048512047E1207021103115012048568
:100E30001206F2202C0312039C302C031203E31140
:100E4000031173120485120702110311981204850D
:100E50001206F2110311BB120485120702110311CD
:100E6000E01204851203F91206F211033103120392
:100E7000FD120485302827855B5979187A0CC3E563
:100E80003999400EC228D2298A3B855B59855B5A25
:100E9000800CC3E55294014003020E26E11E302966
:100EA0001C202B19E53B147006C229D22AC126F555
:100EB0003BC3E55294014003020E268061753C005D
:100EC00078FA79A4E760027803C3E55398504FE5B8
:100ED00023604B303A17203805203407800F303418
:100EE00002800A202B07D22B855B59C15078F03045
:100EF0002B05855B597820C3E548985003020E26E0
:100F0000302B1BC22BC238303402D238D229753B69
:100F100012855B59C126053CE5526002E121753C12
:100F200000C2AF312775240075250075A91375A778
:100F30001075C10075A700756400D2AF12032C3183
:100F40002778A4E66006D291D293D295C3E53C946B
:100F500004400261D3A152901A0D7820F1CCE52013
:100F6000B4550AA3F1CCE520B4AA0280063137F1CA
:100F700091801D901A0378807B0AF1CCA308DBFADC
:100F8000901A0F788C7B1AF1CCA308DBFA901A29FF
:100F900022C2AF12100DF1E5901A007410F1D1A326
:100FA0007401F1D1A37420F1D1901A0378807B0AE7
:100FB000F1D0A308DBFA901A0F788C7B1AF1D0A33A
:100FC00008DBFA121021F1FC901A2922E493F62290
:100FD000E6438F01538FFD75EF0275B7A575B7F125
:100FE000F0538FFE22438F02438F0175EF0275B7D6
:100FF000A575B7F1901A0DF0538FFC22901A0D745D
:1010000055120FD1901A0E74AA120FD1227A30798C
:10101000D07820901A40120FCCE520F709A3DAF619
:10102000227A3079D0901A40E7120FD109A3DAF86A
:10103000227C05120330DCFB22C2AF12033F1203F5
:101040004512034B12035112032412033F120345AE
:1010500012034B12035112032412033F12034512D1
:10106000034B120351D2AF22C2AF12035112034BF2
:1010700012034512033F12032412035112034B12B1
:10108000034512033F12032412035112034B1203B0
:071090004512033FD2AF221D
:1019FD00020B33100120FFFFFFFFFFFF09FF01FF67
:101A0D0055AA01FFFFFFFFFF03FFFFFF25D0285061
:0D1A1D0004FF02FF7AFF0101FFFF0000FF40
:101A400023455F485F3530232020202020202020A0
:101A500023424C48454C492445464D3842323123B7
:101A60002020202020202020202020202020202076
:101C0000C2AFC2D37597DE7597AD7581C075A90057
:101C100043FF80752438752503B1C875EF0243F181
:101C20002053A4DFD28575D4FF75E3407DFA780395
:101C300079E67C10752200752300901DD57B067512
:101C400024987525013085028145208508D8FBD967
:101C5000F9DCF781B7308508D8FBD9F9DCF781B713
:101C6000B188E493A3C39A6004DDC381B7DBDBB121
:101C70007A6002812E7B08E493FAA3B15BDBF87AE9
:101C800030B15B752200752300B17AEAFCEBFDC32D
:101C9000ED94FE400EB17A8A278B28ED30E0048A5D
:101CA000828B83B17A7AC270D8C3ED94FE601350F0
:101CB000CEBD0023EC60097520007521FF020000F5
:101CC0008100A827A9280809D804D90281D4B17EA7
:101CD000EAF281C80D81A3C3ED94035047EDA2E061
:101CE00092007AC5C3E5829400E583941C5092204B
:101CF0000010438F02438F0175B7A575B7F1F0301F
:101D0000001DA827A9280809438F01538FFDD80477
:101D1000D902A11FE275B7A575B7F1F0A3A10E53C3
:101D20008FFC817F7AC1BD030CE493A3FAB13FDC41
:101D3000F8B137817F8181AA22AB23B15BEBFAEA4C
:101D40006222752608C3E52313F523E52213F52245
:101D500050066323A0632201D526EAB1C8B1C87535
:101D6000260AEAF4200102D285300102C285B1C8F8
:101D7000C3134002C201D526EB22B17EEAFB2085C7
:101D800002A17E308502A183752608AE24AF25C34B
:101D9000EF13FFEE13FEB1CCB1C8C3EA13308502D6
:101DA0004480FA30E703632201C3E52313F523E5FA
:101DB0002213F52250066323A0632201D526D9E51C
:101DC0002265236523F52222AE24AF250E0FDEFE09
:101DD000DFFCD20122424C48656C6934373163E83C
:031DE000B2060147
:00000001FF
